Archive member included to satisfy reference by file (symbol)

/usr/local/bin/../lib/gcc/arm-none-eabi/8.3.1/../../../../arm-none-eabi/lib/thumb/v7e-m+fp/hard/libc_nano.a(lib_a-exit.o)
                              /usr/local/bin/../lib/gcc/arm-none-eabi/8.3.1/../../../../arm-none-eabi/lib/thumb/v7e-m+fp/hard/crt0.o (exit)
/usr/local/bin/../lib/gcc/arm-none-eabi/8.3.1/../../../../arm-none-eabi/lib/thumb/v7e-m+fp/hard/libc_nano.a(lib_a-impure.o)
                              /usr/local/bin/../lib/gcc/arm-none-eabi/8.3.1/../../../../arm-none-eabi/lib/thumb/v7e-m+fp/hard/libc_nano.a(lib_a-exit.o) (_global_impure_ptr)
/usr/local/bin/../lib/gcc/arm-none-eabi/8.3.1/../../../../arm-none-eabi/lib/thumb/v7e-m+fp/hard/libc_nano.a(lib_a-init.o)
                              /usr/local/bin/../lib/gcc/arm-none-eabi/8.3.1/../../../../arm-none-eabi/lib/thumb/v7e-m+fp/hard/crt0.o (__libc_init_array)
/usr/local/bin/../lib/gcc/arm-none-eabi/8.3.1/../../../../arm-none-eabi/lib/thumb/v7e-m+fp/hard/libc_nano.a(lib_a-memset.o)
                              /usr/local/bin/../lib/gcc/arm-none-eabi/8.3.1/../../../../arm-none-eabi/lib/thumb/v7e-m+fp/hard/crt0.o (memset)
/usr/local/bin/../lib/gcc/arm-none-eabi/8.3.1/../../../../arm-none-eabi/lib/thumb/v7e-m+fp/hard/libnosys.a(_exit.o)
                              /usr/local/bin/../lib/gcc/arm-none-eabi/8.3.1/../../../../arm-none-eabi/lib/thumb/v7e-m+fp/hard/libc_nano.a(lib_a-exit.o) (_exit)
/usr/local/bin/../lib/gcc/arm-none-eabi/8.3.1/../../../../arm-none-eabi/lib/thumb/v7e-m+fp/hard/libc_nano.a(lib_a-memcpy-stub.o)
                              _build/nrf52832_xxaa_SEGGER_RTT.c.o (memcpy)
/usr/local/bin/../lib/gcc/arm-none-eabi/8.3.1/../../../../arm-none-eabi/lib/thumb/v7e-m+fp/hard/libc_nano.a(lib_a-strcpy.o)
                              _build/nrf52832_xxaa_SEGGER_RTT.c.o (strcpy)
/usr/local/bin/../lib/gcc/arm-none-eabi/8.3.1/../../../../arm-none-eabi/lib/thumb/v7e-m+fp/hard/libc_nano.a(lib_a-strlen.o)
                              _build/nrf52832_xxaa_SEGGER_RTT.c.o (strlen)

Allocating common symbols
Common symbol       size              file

_SEGGER_RTT         0x78              _build/nrf52832_xxaa_SEGGER_RTT.c.o

Discarded input sections

 .text          0x0000000000000000        0x0 /usr/local/bin/../lib/gcc/arm-none-eabi/8.3.1/thumb/v7e-m+fp/hard/crti.o
 .data          0x0000000000000000        0x0 /usr/local/bin/../lib/gcc/arm-none-eabi/8.3.1/thumb/v7e-m+fp/hard/crti.o
 .bss           0x0000000000000000        0x0 /usr/local/bin/../lib/gcc/arm-none-eabi/8.3.1/thumb/v7e-m+fp/hard/crti.o
 .data          0x0000000000000000        0x4 /usr/local/bin/../lib/gcc/arm-none-eabi/8.3.1/thumb/v7e-m+fp/hard/crtbegin.o
 .data          0x0000000000000000        0x0 /usr/local/bin/../lib/gcc/arm-none-eabi/8.3.1/../../../../arm-none-eabi/lib/thumb/v7e-m+fp/hard/crt0.o
 .bss           0x0000000000000000        0x0 /usr/local/bin/../lib/gcc/arm-none-eabi/8.3.1/../../../../arm-none-eabi/lib/thumb/v7e-m+fp/hard/crt0.o
 .ARM.extab     0x0000000000000000        0x0 /usr/local/bin/../lib/gcc/arm-none-eabi/8.3.1/../../../../arm-none-eabi/lib/thumb/v7e-m+fp/hard/crt0.o
 .text          0x0000000000000000        0x0 /usr/local/bin/../lib/gcc/arm-none-eabi/8.3.1/../../../../arm-none-eabi/lib/thumb/v7e-m+fp/hard/libc_nano.a(lib_a-exit.o)
 .data          0x0000000000000000        0x0 /usr/local/bin/../lib/gcc/arm-none-eabi/8.3.1/../../../../arm-none-eabi/lib/thumb/v7e-m+fp/hard/libc_nano.a(lib_a-exit.o)
 .bss           0x0000000000000000        0x0 /usr/local/bin/../lib/gcc/arm-none-eabi/8.3.1/../../../../arm-none-eabi/lib/thumb/v7e-m+fp/hard/libc_nano.a(lib_a-exit.o)
 .text          0x0000000000000000        0x0 /usr/local/bin/../lib/gcc/arm-none-eabi/8.3.1/../../../../arm-none-eabi/lib/thumb/v7e-m+fp/hard/libc_nano.a(lib_a-impure.o)
 .data          0x0000000000000000        0x0 /usr/local/bin/../lib/gcc/arm-none-eabi/8.3.1/../../../../arm-none-eabi/lib/thumb/v7e-m+fp/hard/libc_nano.a(lib_a-impure.o)
 .bss           0x0000000000000000        0x0 /usr/local/bin/../lib/gcc/arm-none-eabi/8.3.1/../../../../arm-none-eabi/lib/thumb/v7e-m+fp/hard/libc_nano.a(lib_a-impure.o)
 .data._impure_ptr
                0x0000000000000000        0x4 /usr/local/bin/../lib/gcc/arm-none-eabi/8.3.1/../../../../arm-none-eabi/lib/thumb/v7e-m+fp/hard/libc_nano.a(lib_a-impure.o)
 .text          0x0000000000000000        0x0 /usr/local/bin/../lib/gcc/arm-none-eabi/8.3.1/../../../../arm-none-eabi/lib/thumb/v7e-m+fp/hard/libc_nano.a(lib_a-init.o)
 .data          0x0000000000000000        0x0 /usr/local/bin/../lib/gcc/arm-none-eabi/8.3.1/../../../../arm-none-eabi/lib/thumb/v7e-m+fp/hard/libc_nano.a(lib_a-init.o)
 .bss           0x0000000000000000        0x0 /usr/local/bin/../lib/gcc/arm-none-eabi/8.3.1/../../../../arm-none-eabi/lib/thumb/v7e-m+fp/hard/libc_nano.a(lib_a-init.o)
Memory Configuration

Name             Origin             Length             Attributes
FLASH            0x0000000000000000 0x0000000000080000 xr
RAM              0x0000000020000000 0x0000000000010000 xrw
*default*        0x0000000000000000 0xffffffffffffffff

Linker script and memory map


.text           0x0000000000000000      0xd48
 *(.isr_vector)
 .isr_vector    0x0000000000000000      0x200 _build/nrf52832_xxaa_gcc_startup_nrf52.S.o
                0x0000000000000000                __isr_vector
 *(.text*)
 .text          0x0000000000000200       0x40 /usr/local/bin/../lib/gcc/arm-none-eabi/8.3.1/thumb/v7e-m+fp/hard/crtbegin.o
 .text          0x0000000000000240       0x74 /usr/local/bin/../lib/gcc/arm-none-eabi/8.3.1/../../../../arm-none-eabi/lib/thumb/v7e-m+fp/hard/crt0.o
                0x0000000000000240                _mainCRTStartup
                0x0000000000000240                _start
 .text.exit     0x00000000000002b4       0x28 /usr/local/bin/../lib/gcc/arm-none-eabi/8.3.1/../../../../arm-none-eabi/lib/thumb/v7e-m+fp/hard/libc_nano.a(lib_a-exit.o)
                0x00000000000002b4                exit
 .text.__libc_init_array
                0x00000000000002dc       0x48 /usr/local/bin/../lib/gcc/arm-none-eabi/8.3.1/../../../../arm-none-eabi/lib/thumb/v7e-m+fp/hard/libc_nano.a(lib_a-init.o)
                0x00000000000002dc                __libc_init_array
 .text.memset   0x0000000000000324       0x10 /usr/local/bin/../lib/gcc/arm-none-eabi/8.3.1/../../../../arm-none-eabi/lib/thumb/v7e-m+fp/hard/libc_nano.a(lib_a-memset.o)
                0x0000000000000324                memset
 .text._exit    0x0000000000000334        0x4 /usr/local/bin/../lib/gcc/arm-none-eabi/8.3.1/../../../../arm-none-eabi/lib/thumb/v7e-m+fp/hard/libnosys.a(_exit.o)
                0x0000000000000334                _exit
 .text.startup.main
                0x0000000000000338       0x44 _build/nrf52832_xxaa_main.c.o
                0x0000000000000338                main
 .text.init_LED1
                0x000000000000037c        0xc _build/nrf52832_xxaa_gpio.c.o
                0x000000000000037c                init_LED1
 .text.turnON_LED1
                0x0000000000000388       0x10 _build/nrf52832_xxaa_gpio.c.o
                0x0000000000000388                turnON_LED1
 .text.turnOFF_LED1
                0x0000000000000398       0x10 _build/nrf52832_xxaa_gpio.c.o
                0x0000000000000398                turnOFF_LED1
 .text.GPIOTE_IRQHandler
                0x00000000000003a8      0x2d4 _build/nrf52832_xxaa_nrf_drv_gpiote.c.o
                0x00000000000003a8                GPIOTE_IRQHandler
 .text.TIMER0_IRQHandler
                0x000000000000067c       0x58 _build/nrf52832_xxaa_nrf_drv_timer.c.o
                0x000000000000067c                TIMER0_IRQHandler
 .text.UARTE0_UART0_IRQHandler
                0x00000000000006d4      0x2dc _build/nrf52832_xxaa_nrf_drv_uart.c.o
                0x00000000000006d4                UARTE0_UART0_IRQHandler
 .text          0x00000000000009b0       0x3c _build/nrf52832_xxaa_gcc_startup_nrf52.S.o
                0x00000000000009b0                Reset_Handler
                0x00000000000009d8                NMI_Handler
                0x00000000000009da                HardFault_Handler
                0x00000000000009dc                MemoryManagement_Handler
                0x00000000000009de                BusFault_Handler
                0x00000000000009e0                UsageFault_Handler
                0x00000000000009e2                SVC_Handler
                0x00000000000009e4                DebugMon_Handler
                0x00000000000009e6                PendSV_Handler
                0x00000000000009e8                SysTick_Handler
                0x00000000000009ea                TIMER2_IRQHandler
                0x00000000000009ea                RTC0_IRQHandler
                0x00000000000009ea                SWI0_EGU0_IRQHandler
                0x00000000000009ea                SWI2_EGU2_IRQHandler
                0x00000000000009ea                PWM1_IRQHandler
                0x00000000000009ea                POWER_CLOCK_IRQHandler
                0x00000000000009ea                RADIO_IRQHandler
                0x00000000000009ea                PDM_IRQHandler
                0x00000000000009ea                TEMP_IRQHandler
                0x00000000000009ea                QDEC_IRQHandler
                0x00000000000009ea                TIMER3_IRQHandler
                0x00000000000009ea                FPU_IRQHandler
                0x00000000000009ea                SPIM0_SPIS0_TWIM0_TWIS0_SPI0_TWI0_IRQHandler
                0x00000000000009ea                TIMER4_IRQHandler
                0x00000000000009ea                I2S_IRQHandler
                0x00000000000009ea                SWI4_EGU4_IRQHandler
                0x00000000000009ea                TIMER1_IRQHandler
                0x00000000000009ea                PWM2_IRQHandler
                0x00000000000009ea                ECB_IRQHandler
                0x00000000000009ea                SPIM1_SPIS1_TWIM1_TWIS1_SPI1_TWI1_IRQHandler
                0x00000000000009ea                Default_Handler
                0x00000000000009ea                SAADC_IRQHandler
                0x00000000000009ea                CCM_AAR_IRQHandler
                0x00000000000009ea                WDT_IRQHandler
                0x00000000000009ea                SWI5_EGU5_IRQHandler
                0x00000000000009ea                RNG_IRQHandler
                0x00000000000009ea                RTC2_IRQHandler
                0x00000000000009ea                PWM0_IRQHandler
                0x00000000000009ea                SWI3_EGU3_IRQHandler
                0x00000000000009ea                RTC1_IRQHandler
                0x00000000000009ea                SWI1_EGU1_IRQHandler
                0x00000000000009ea                SPIM2_SPIS2_SPI2_IRQHandler
                0x00000000000009ea                NFCT_IRQHandler
                0x00000000000009ea                MWU_IRQHandler
                0x00000000000009ea                COMP_LPCOMP_IRQHandler
 .text.SystemInit
                0x00000000000009ec      0x33c _build/nrf52832_xxaa_system_nrf52.c.o
                0x00000000000009ec                SystemInit
 *(.init)
 .init          0x0000000000000d28        0x4 /usr/local/bin/../lib/gcc/arm-none-eabi/8.3.1/thumb/v7e-m+fp/hard/crti.o
                0x0000000000000d28                _init
 .init          0x0000000000000d2c        0x8 /usr/local/bin/../lib/gcc/arm-none-eabi/8.3.1/thumb/v7e-m+fp/hard/crtn.o
 *(.fini)
 .fini          0x0000000000000d34        0x4 /usr/local/bin/../lib/gcc/arm-none-eabi/8.3.1/thumb/v7e-m+fp/hard/crti.o
                0x0000000000000d34                _fini
 .fini          0x0000000000000d38        0x8 /usr/local/bin/../lib/gcc/arm-none-eabi/8.3.1/thumb/v7e-m+fp/hard/crtn.o
 *crtbegin.o(.ctors)
 *crtbegin?.o(.ctors)
 *(EXCLUDE_FILE(*crtend.o *crtend?.o) .ctors)
 *(SORT_BY_NAME(.ctors.*))
 *(.ctors)
 *crtbegin.o(.dtors)
 *crtbegin?.o(.dtors)
 *(EXCLUDE_FILE(*crtend.o *crtend?.o) .dtors)
 *(SORT_BY_NAME(.dtors.*))
 *(.dtors)
 *(.rodata*)
 .rodata._global_impure_ptr
                0x0000000000000d40        0x4 /usr/local/bin/../lib/gcc/arm-none-eabi/8.3.1/../../../../arm-none-eabi/lib/thumb/v7e-m+fp/hard/libc_nano.a(lib_a-impure.o)
                0x0000000000000d40                _global_impure_ptr
 *(.eh_frame*)
 .eh_frame      0x0000000000000d44        0x0 /usr/local/bin/../lib/gcc/arm-none-eabi/8.3.1/thumb/v7e-m+fp/hard/crtbegin.o
 .eh_frame      0x0000000000000d44        0x4 /usr/local/bin/../lib/gcc/arm-none-eabi/8.3.1/thumb/v7e-m+fp/hard/crtend.o

.glue_7         0x0000000000000d48        0x0
 .glue_7        0x0000000000000d48        0x0 linker stubs

.glue_7t        0x0000000000000d48        0x0
 .glue_7t       0x0000000000000d48        0x0 linker stubs

.vfp11_veneer   0x0000000000000d48        0x0
 .vfp11_veneer  0x0000000000000d48        0x0 linker stubs

.v4_bx          0x0000000000000d48        0x0
 .v4_bx         0x0000000000000d48        0x0 linker stubs

.iplt           0x0000000000000d48        0x0
 .iplt          0x0000000000000d48        0x0 /usr/local/bin/../lib/gcc/arm-none-eabi/8.3.1/thumb/v7e-m+fp/hard/crtbegin.o

.pwr_mgmt_data  0x0000000000000d48        0x0
                [!provide]                        PROVIDE (__start_pwr_mgmt_data = .)
 *(SORT_BY_NAME(.pwr_mgmt_data*))
                [!provide]                        PROVIDE (__stop_pwr_mgmt_data = .)

.ARM.extab
 *(.ARM.extab* .gnu.linkonce.armextab.*)
                0x0000000000000d48                __exidx_start = .

.ARM.exidx      0x0000000000000d48        0x8
 *(.ARM.exidx* .gnu.linkonce.armexidx.*)
 .ARM.exidx     0x0000000000000d48        0x8 /usr/local/bin/../lib/gcc/arm-none-eabi/8.3.1/../../../../arm-none-eabi/lib/thumb/v7e-m+fp/hard/crt0.o
                0x0000000000000d50                __exidx_end = .
                0x0000000000000d50                __etext = .

.rel.dyn        0x0000000000000d50        0x0
 .rel.iplt      0x0000000000000d50        0x0 /usr/local/bin/../lib/gcc/arm-none-eabi/8.3.1/thumb/v7e-m+fp/hard/crtbegin.o

.data           0x0000000020000000       0x6c load address 0x0000000000000d50
                0x0000000020000000                __data_start__ = .
 *(vtable)
 *(.data*)
 .data.impure_data
                0x0000000020000000       0x60 /usr/local/bin/../lib/gcc/arm-none-eabi/8.3.1/../../../../arm-none-eabi/lib/thumb/v7e-m+fp/hard/libc_nano.a(lib_a-impure.o)
 .data.SystemCoreClock
                0x0000000020000060        0x4 _build/nrf52832_xxaa_system_nrf52.c.o
                0x0000000020000060                SystemCoreClock
                0x0000000020000064                . = ALIGN (0x4)
                0x0000000020000064                PROVIDE (__preinit_array_start = .)
 *(.preinit_array)
                0x0000000020000064                PROVIDE (__preinit_array_end = .)
                0x0000000020000064                . = ALIGN (0x4)
                0x0000000020000064                PROVIDE (__init_array_start = .)
 *(SORT_BY_NAME(.init_array.*))
 *(.init_array)
 .init_array    0x0000000020000064        0x4 /usr/local/bin/../lib/gcc/arm-none-eabi/8.3.1/thumb/v7e-m+fp/hard/crtbegin.o
                0x0000000020000068                PROVIDE (__init_array_end = .)
                0x0000000020000068                . = ALIGN (0x4)
                [!provide]                        PROVIDE (__fini_array_start = .)
 *(SORT_BY_NAME(.fini_array.*))
 *(.fini_array)
 .fini_array    0x0000000020000068        0x4 /usr/local/bin/../lib/gcc/arm-none-eabi/8.3.1/thumb/v7e-m+fp/hard/crtbegin.o
                [!provide]                        PROVIDE (__fini_array_end = .)
 *(.jcr*)
                0x000000002000006c                . = ALIGN (0x4)
                0x000000002000006c                __data_end__ = .
LOAD /usr/local/bin/../lib/gcc/arm-none-eabi/8.3.1/thumb/v7e-m+fp/hard/crti.o
LOAD /usr/local/bin/../lib/gcc/arm-none-eabi/8.3.1/thumb/v7e-m+fp/hard/crtbegin.o
LOAD /usr/local/bin/../lib/gcc/arm-none-eabi/8.3.1/../../../../arm-none-eabi/lib/thumb/v7e-m+fp/hard/crt0.o
LOAD /usr/local/bin/../lib/gcc/arm-none-eabi/8.3.1/../../../../arm-none-eabi/lib/thumb/v7e-m+fp/hard/libc_nano.a
LOAD /usr/local/bin/../lib/gcc/arm-none-eabi/8.3.1/../../../../arm-none-eabi/lib/thumb/v7e-m+fp/hard/libnosys.a
LOAD _build/nrf52832_xxaa_main.c.o
LOAD _build/nrf52832_xxaa_gpio.c.o
LOAD _build/nrf52832_xxaa_nrf_log_backend_serial.c.o
LOAD _build/nrf52832_xxaa_nrf_log_frontend.c.o
LOAD _build/nrf52832_xxaa_boards.c.o
LOAD _build/nrf52832_xxaa_app_error.c.o
LOAD _build/nrf52832_xxaa_app_error_weak.c.o
LOAD _build/nrf52832_xxaa_app_util_platform.c.o
LOAD _build/nrf52832_xxaa_nrf_assert.c.o
LOAD _build/nrf52832_xxaa_nrf_strerror.c.o
LOAD _build/nrf52832_xxaa_nrf_drv_common.c.o
LOAD _build/nrf52832_xxaa_nrf_drv_gpiote.c.o
LOAD _build/nrf52832_xxaa_nrf_drv_ppi.c.o
LOAD _build/nrf52832_xxaa_nrf_drv_timer.c.o
LOAD _build/nrf52832_xxaa_nrf_drv_uart.c.o
LOAD _build/nrf52832_xxaa_RTT_Syscalls_GCC.c.o
LOAD _build/nrf52832_xxaa_SEGGER_RTT.c.o
LOAD _build/nrf52832_xxaa_SEGGER_RTT_printf.c.o
LOAD _build/nrf52832_xxaa_gcc_startup_nrf52.S.o
LOAD _build/nrf52832_xxaa_system_nrf52.c.o
LOAD /usr/local/bin/../lib/gcc/arm-none-eabi/8.3.1/../../../../arm-none-eabi/lib/thumb/v7e-m+fp/hard/libm.a
START GROUP
LOAD /usr/local/bin/../lib/gcc/arm-none-eabi/8.3.1/thumb/v7e-m+fp/hard/libgcc.a
LOAD /usr/local/bin/../lib/gcc/arm-none-eabi/8.3.1/../../../../arm-none-eabi/lib/thumb/v7e-m+fp/hard/libc_nano.a
END GROUP
START GROUP
LOAD /usr/local/bin/../lib/gcc/arm-none-eabi/8.3.1/thumb/v7e-m+fp/hard/libgcc.a
LOAD /usr/local/bin/../lib/gcc/arm-none-eabi/8.3.1/../../../../arm-none-eabi/lib/thumb/v7e-m+fp/hard/libc_nano.a
END GROUP
LOAD /usr/local/bin/../lib/gcc/arm-none-eabi/8.3.1/thumb/v7e-m+fp/hard/crtend.o
LOAD /usr/local/bin/../lib/gcc/arm-none-eabi/8.3.1/thumb/v7e-m+fp/hard/crtn.o
START GROUP
LOAD /usr/local/bin/../lib/gcc/arm-none-eabi/8.3.1/thumb/v7e-m+fp/hard/libgcc.a
LOAD /usr/local/bin/../lib/gcc/arm-none-eabi/8.3.1/../../../../arm-none-eabi/lib/thumb/v7e-m+fp/hard/libc.a
LOAD /usr/local/bin/../lib/gcc/arm-none-eabi/8.3.1/../../../../arm-none-eabi/lib/thumb/v7e-m+fp/hard/libnosys.a
END GROUP

.igot.plt       0x000000002000006c        0x0 load address 0x0000000000000dbc
 .igot.plt      0x000000002000006c        0x0 /usr/local/bin/../lib/gcc/arm-none-eabi/8.3.1/thumb/v7e-m+fp/hard/crtbegin.o

.fs_data        0x000000002000006c        0x0
                [!provide]                        PROVIDE (__start_fs_data = .)
 *(.fs_data)
                [!provide]                        PROVIDE (__stop_fs_data = .)

.bss            0x0000000020000070       0x94 load address 0x0000000000000dc0
                0x0000000020000070                . = ALIGN (0x4)
                0x0000000020000070                __bss_start__ = .
 *(.bss*)
 .bss           0x0000000020000070       0x1c /usr/local/bin/../lib/gcc/arm-none-eabi/8.3.1/thumb/v7e-m+fp/hard/crtbegin.o
 *fill*         0x000000002000008c        0x4 
 .bss.m_cb      0x0000000020000090       0x48 _build/nrf52832_xxaa_nrf_drv_gpiote.c.o
 .bss.m_cb      0x00000000200000d8        0xc _build/nrf52832_xxaa_nrf_drv_timer.c.o
 .bss.m_cb      0x00000000200000e4       0x20 _build/nrf52832_xxaa_nrf_drv_uart.c.o
 *(COMMON)
                0x0000000020000104                . = ALIGN (0x4)
                0x0000000020000104                __bss_end__ = .

.heap           0x0000000020000108     0x2000
                0x0000000020000108                __HeapBase = .
                0x0000000020000108                __end__ = .
                [!provide]                        PROVIDE (end = .)
 *(.heap*)
 .heap          0x0000000020000108     0x2000 _build/nrf52832_xxaa_gcc_startup_nrf52.S.o
                0x0000000020002108                __HeapLimit = .

.stack_dummy    0x0000000020000108     0x2000
 *(.stack*)
 .stack         0x0000000020000108     0x2000 _build/nrf52832_xxaa_gcc_startup_nrf52.S.o
                0x0000000020010000                __StackTop = (ORIGIN (RAM) + LENGTH (RAM))
                0x000000002000e000                __StackLimit = (__StackTop - SIZEOF (.stack_dummy))
                0x0000000020010000                PROVIDE (__stack = __StackTop)
                0x0000000000000001                ASSERT ((__StackLimit >= __HeapLimit), region RAM overflowed with stack)
OUTPUT(_build/nrf52832_xxaa.out elf32-littlearm)

.ARM.attributes
                0x0000000000000000       0x30
 .ARM.attributes
                0x0000000000000000       0x1e /usr/local/bin/../lib/gcc/arm-none-eabi/8.3.1/thumb/v7e-m+fp/hard/crti.o
 .ARM.attributes
                0x000000000000001e       0x34 /usr/local/bin/../lib/gcc/arm-none-eabi/8.3.1/thumb/v7e-m+fp/hard/crtbegin.o
 .ARM.attributes
                0x0000000000000052       0x1c /usr/local/bin/../lib/gcc/arm-none-eabi/8.3.1/../../../../arm-none-eabi/lib/thumb/v7e-m+fp/hard/crt0.o
 .ARM.attributes
                0x000000000000006e       0x34 /usr/local/bin/../lib/gcc/arm-none-eabi/8.3.1/../../../../arm-none-eabi/lib/thumb/v7e-m+fp/hard/libc_nano.a(lib_a-exit.o)
 .ARM.attributes
                0x00000000000000a2       0x32 /usr/local/bin/../lib/gcc/arm-none-eabi/8.3.1/../../../../arm-none-eabi/lib/thumb/v7e-m+fp/hard/libc_nano.a(lib_a-impure.o)
 .ARM.attributes
                0x00000000000000d4       0x34 /usr/local/bin/../lib/gcc/arm-none-eabi/8.3.1/../../../../arm-none-eabi/lib/thumb/v7e-m+fp/hard/libc_nano.a(lib_a-init.o)
 .ARM.attributes
                0x0000000000000108       0x34 /usr/local/bin/../lib/gcc/arm-none-eabi/8.3.1/../../../../arm-none-eabi/lib/thumb/v7e-m+fp/hard/libc_nano.a(lib_a-memset.o)
 .ARM.attributes
                0x000000000000013c       0x34 /usr/local/bin/../lib/gcc/arm-none-eabi/8.3.1/../../../../arm-none-eabi/lib/thumb/v7e-m+fp/hard/libnosys.a(_exit.o)
 .ARM.attributes
                0x0000000000000170       0x34 _build/nrf52832_xxaa_main.c.o
 .ARM.attributes
                0x00000000000001a4       0x34 _build/nrf52832_xxaa_gpio.c.o
 .ARM.attributes
                0x00000000000001d8       0x34 _build/nrf52832_xxaa_nrf_drv_gpiote.c.o
 .ARM.attributes
                0x000000000000020c       0x34 _build/nrf52832_xxaa_nrf_drv_timer.c.o
 .ARM.attributes
                0x0000000000000240       0x34 _build/nrf52832_xxaa_nrf_drv_uart.c.o
 .ARM.attributes
                0x0000000000000274       0x1c _build/nrf52832_xxaa_gcc_startup_nrf52.S.o
 .ARM.attributes
                0x0000000000000290       0x34 _build/nrf52832_xxaa_system_nrf52.c.o
 .ARM.attributes
                0x00000000000002c4       0x32 /usr/local/bin/../lib/gcc/arm-none-eabi/8.3.1/thumb/v7e-m+fp/hard/crtend.o
 .ARM.attributes
                0x00000000000002f6       0x1e /usr/local/bin/../lib/gcc/arm-none-eabi/8.3.1/thumb/v7e-m+fp/hard/crtn.o

.comment        0x0000000000000000       0x76
 .comment       0x0000000000000000       0x76 _build/nrf52832_xxaa_main.c.o
                                         0x77 (size before relaxing)
 .comment       0x0000000000000076       0x77 _build/nrf52832_xxaa_gpio.c.o
 .comment       0x0000000000000076       0x77 _build/nrf52832_xxaa_nrf_drv_gpiote.c.o
 .comment       0x0000000000000076       0x77 _build/nrf52832_xxaa_nrf_drv_timer.c.o
 .comment       0x0000000000000076       0x77 _build/nrf52832_xxaa_nrf_drv_uart.c.o
 .comment       0x0000000000000076       0x77 _build/nrf52832_xxaa_system_nrf52.c.o

.debug_frame    0x0000000000000000      0x71c
 .debug_frame   0x0000000000000000       0x28 /usr/local/bin/../lib/gcc/arm-none-eabi/8.3.1/../../../../arm-none-eabi/lib/thumb/v7e-m+fp/hard/libc_nano.a(lib_a-exit.o)
 .debug_frame   0x0000000000000028       0x2c /usr/local/bin/../lib/gcc/arm-none-eabi/8.3.1/../../../../arm-none-eabi/lib/thumb/v7e-m+fp/hard/libc_nano.a(lib_a-init.o)
 .debug_frame   0x0000000000000054       0x20 /usr/local/bin/../lib/gcc/arm-none-eabi/8.3.1/../../../../arm-none-eabi/lib/thumb/v7e-m+fp/hard/libc_nano.a(lib_a-memset.o)
 .debug_frame   0x0000000000000074       0x20 /usr/local/bin/../lib/gcc/arm-none-eabi/8.3.1/../../../../arm-none-eabi/lib/thumb/v7e-m+fp/hard/libnosys.a(_exit.o)
 .debug_frame   0x0000000000000094       0x28 _build/nrf52832_xxaa_main.c.o
 .debug_frame   0x00000000000000bc       0x40 _build/nrf52832_xxaa_gpio.c.o
 .debug_frame   0x00000000000000fc      0x294 _build/nrf52832_xxaa_nrf_drv_gpiote.c.o
 .debug_frame   0x0000000000000390      0x178 _build/nrf52832_xxaa_nrf_drv_timer.c.o
 .debug_frame   0x0000000000000508      0x1d4 _build/nrf52832_xxaa_nrf_drv_uart.c.o
 .debug_frame   0x00000000000006dc       0x40 _build/nrf52832_xxaa_system_nrf52.c.o

.debug_info     0x0000000000000000     0xd62d
 .debug_info    0x0000000000000000      0x9cc _build/nrf52832_xxaa_main.c.o
 .debug_info    0x00000000000009cc      0xab5 _build/nrf52832_xxaa_gpio.c.o
 .debug_info    0x0000000000001481     0x37dd _build/nrf52832_xxaa_nrf_drv_gpiote.c.o
 .debug_info    0x0000000000004c5e     0x217f _build/nrf52832_xxaa_nrf_drv_timer.c.o
 .debug_info    0x0000000000006ddd     0x5954 _build/nrf52832_xxaa_nrf_drv_uart.c.o
 .debug_info    0x000000000000c731      0xefc _build/nrf52832_xxaa_system_nrf52.c.o

.debug_abbrev   0x0000000000000000     0x15c3
 .debug_abbrev  0x0000000000000000      0x20c _build/nrf52832_xxaa_main.c.o
 .debug_abbrev  0x000000000000020c      0x200 _build/nrf52832_xxaa_gpio.c.o
 .debug_abbrev  0x000000000000040c      0x597 _build/nrf52832_xxaa_nrf_drv_gpiote.c.o
 .debug_abbrev  0x00000000000009a3      0x4e6 _build/nrf52832_xxaa_nrf_drv_timer.c.o
 .debug_abbrev  0x0000000000000e89      0x514 _build/nrf52832_xxaa_nrf_drv_uart.c.o
 .debug_abbrev  0x000000000000139d      0x226 _build/nrf52832_xxaa_system_nrf52.c.o

.debug_aranges  0x0000000000000000      0x250
 .debug_aranges
                0x0000000000000000       0x20 _build/nrf52832_xxaa_main.c.o
 .debug_aranges
                0x0000000000000020       0x30 _build/nrf52832_xxaa_gpio.c.o
 .debug_aranges
                0x0000000000000050       0xd8 _build/nrf52832_xxaa_nrf_drv_gpiote.c.o
 .debug_aranges
                0x0000000000000128       0x88 _build/nrf52832_xxaa_nrf_drv_timer.c.o
 .debug_aranges
                0x00000000000001b0       0x78 _build/nrf52832_xxaa_nrf_drv_uart.c.o
 .debug_aranges
                0x0000000000000228       0x28 _build/nrf52832_xxaa_system_nrf52.c.o

.debug_ranges   0x0000000000000000     0x2250
 .debug_ranges  0x0000000000000000       0x10 _build/nrf52832_xxaa_main.c.o
 .debug_ranges  0x0000000000000010       0x20 _build/nrf52832_xxaa_gpio.c.o
 .debug_ranges  0x0000000000000030     0x1118 _build/nrf52832_xxaa_nrf_drv_gpiote.c.o
 .debug_ranges  0x0000000000001148      0x310 _build/nrf52832_xxaa_nrf_drv_timer.c.o
 .debug_ranges  0x0000000000001458      0xc38 _build/nrf52832_xxaa_nrf_drv_uart.c.o
 .debug_ranges  0x0000000000002090      0x1c0 _build/nrf52832_xxaa_system_nrf52.c.o

.debug_macro    0x0000000000000000    0x12601
 .debug_macro   0x0000000000000000      0x290 _build/nrf52832_xxaa_main.c.o
 .debug_macro   0x0000000000000290      0xae4 _build/nrf52832_xxaa_main.c.o
 .debug_macro   0x0000000000000d74       0x2d _build/nrf52832_xxaa_main.c.o
 .debug_macro   0x0000000000000da1       0x22 _build/nrf52832_xxaa_main.c.o
 .debug_macro   0x0000000000000dc3       0x56 _build/nrf52832_xxaa_main.c.o
 .debug_macro   0x0000000000000e19       0x51 _build/nrf52832_xxaa_main.c.o
 .debug_macro   0x0000000000000e6a      0x103 _build/nrf52832_xxaa_main.c.o
 .debug_macro   0x0000000000000f6d       0x6a _build/nrf52832_xxaa_main.c.o
 .debug_macro   0x0000000000000fd7      0x1df _build/nrf52832_xxaa_main.c.o
 .debug_macro   0x00000000000011b6       0x35 _build/nrf52832_xxaa_main.c.o
 .debug_macro   0x00000000000011eb       0x50 _build/nrf52832_xxaa_main.c.o
 .debug_macro   0x000000000000123b      0xe66 _build/nrf52832_xxaa_main.c.o
 .debug_macro   0x00000000000020a1      0x392 _build/nrf52832_xxaa_main.c.o
 .debug_macro   0x0000000000002433     0xcc8d _build/nrf52832_xxaa_main.c.o
 .debug_macro   0x000000000000f0c0       0xdc _build/nrf52832_xxaa_main.c.o
 .debug_macro   0x000000000000f19c       0x22 _build/nrf52832_xxaa_main.c.o
 .debug_macro   0x000000000000f1be     0x1313 _build/nrf52832_xxaa_main.c.o
 .debug_macro   0x00000000000104d1       0x82 _build/nrf52832_xxaa_main.c.o
 .debug_macro   0x0000000000010553       0x22 _build/nrf52832_xxaa_main.c.o
 .debug_macro   0x0000000000010575      0x2a4 _build/nrf52832_xxaa_main.c.o
 .debug_macro   0x0000000000010819       0x5e _build/nrf52832_xxaa_main.c.o
 .debug_macro   0x0000000000010877       0x18 _build/nrf52832_xxaa_main.c.o
 .debug_macro   0x000000000001088f       0x35 _build/nrf52832_xxaa_main.c.o
 .debug_macro   0x00000000000108c4       0x34 _build/nrf52832_xxaa_main.c.o
 .debug_macro   0x00000000000108f8       0x16 _build/nrf52832_xxaa_main.c.o
 .debug_macro   0x000000000001090e       0x97 _build/nrf52832_xxaa_main.c.o
 .debug_macro   0x00000000000109a5      0x35c _build/nrf52832_xxaa_main.c.o
 .debug_macro   0x0000000000010d01       0xf6 _build/nrf52832_xxaa_main.c.o
 .debug_macro   0x0000000000010df7       0x10 _build/nrf52832_xxaa_main.c.o
 .debug_macro   0x0000000000010e07       0x16 _build/nrf52832_xxaa_main.c.o
 .debug_macro   0x0000000000010e1d       0x43 _build/nrf52832_xxaa_main.c.o
 .debug_macro   0x0000000000010e60       0x34 _build/nrf52832_xxaa_main.c.o
 .debug_macro   0x0000000000010e94       0x10 _build/nrf52832_xxaa_main.c.o
 .debug_macro   0x0000000000010ea4       0x58 _build/nrf52832_xxaa_main.c.o
 .debug_macro   0x0000000000010efc      0x182 _build/nrf52832_xxaa_main.c.o
 .debug_macro   0x000000000001107e       0xbe _build/nrf52832_xxaa_main.c.o
 .debug_macro   0x000000000001113c       0x16 _build/nrf52832_xxaa_main.c.o
 .debug_macro   0x0000000000011152      0x129 _build/nrf52832_xxaa_main.c.o
 .debug_macro   0x000000000001127b       0x22 _build/nrf52832_xxaa_main.c.o
 .debug_macro   0x000000000001129d       0x8e _build/nrf52832_xxaa_main.c.o
 .debug_macro   0x000000000001132b      0x147 _build/nrf52832_xxaa_main.c.o
 .debug_macro   0x0000000000011472       0x78 _build/nrf52832_xxaa_main.c.o
 .debug_macro   0x00000000000114ea      0x16d _build/nrf52832_xxaa_main.c.o
 .debug_macro   0x0000000000011657       0x2b _build/nrf52832_xxaa_main.c.o
 .debug_macro   0x0000000000011682       0x10 _build/nrf52832_xxaa_main.c.o
 .debug_macro   0x0000000000011692       0x16 _build/nrf52832_xxaa_main.c.o
 .debug_macro   0x00000000000116a8       0x35 _build/nrf52832_xxaa_main.c.o
 .debug_macro   0x00000000000116dd       0x22 _build/nrf52832_xxaa_main.c.o
 .debug_macro   0x00000000000116ff       0x16 _build/nrf52832_xxaa_main.c.o
 .debug_macro   0x0000000000011715      0x296 _build/nrf52832_xxaa_gpio.c.o
 .debug_macro   0x00000000000119ab      0x385 _build/nrf52832_xxaa_nrf_drv_gpiote.c.o
 .debug_macro   0x0000000000011d30       0x1f _build/nrf52832_xxaa_nrf_drv_gpiote.c.o
 .debug_macro   0x0000000000011d4f       0x30 _build/nrf52832_xxaa_nrf_drv_gpiote.c.o
 .debug_macro   0x0000000000011d7f       0x28 _build/nrf52832_xxaa_nrf_drv_gpiote.c.o
 .debug_macro   0x0000000000011da7       0x16 _build/nrf52832_xxaa_nrf_drv_gpiote.c.o
 .debug_macro   0x0000000000011dbd       0x1c _build/nrf52832_xxaa_nrf_drv_gpiote.c.o
 .debug_macro   0x0000000000011dd9      0x31e _build/nrf52832_xxaa_nrf_drv_timer.c.o
 .debug_macro   0x00000000000120f7       0x1c _build/nrf52832_xxaa_nrf_drv_timer.c.o
 .debug_macro   0x0000000000012113       0x34 _build/nrf52832_xxaa_nrf_drv_timer.c.o
 .debug_macro   0x0000000000012147      0x372 _build/nrf52832_xxaa_nrf_drv_uart.c.o
 .debug_macro   0x00000000000124b9       0x10 _build/nrf52832_xxaa_nrf_drv_uart.c.o
 .debug_macro   0x00000000000124c9       0x43 _build/nrf52832_xxaa_nrf_drv_uart.c.o
 .debug_macro   0x000000000001250c       0xf5 _build/nrf52832_xxaa_system_nrf52.c.o

.debug_line     0x0000000000000000     0x6a07
 .debug_line    0x0000000000000000      0x526 _build/nrf52832_xxaa_main.c.o
 .debug_line    0x0000000000000526      0x50c _build/nrf52832_xxaa_gpio.c.o
 .debug_line    0x0000000000000a32     0x230e _build/nrf52832_xxaa_nrf_drv_gpiote.c.o
 .debug_line    0x0000000000002d40      0xecd _build/nrf52832_xxaa_nrf_drv_timer.c.o
 .debug_line    0x0000000000003c0d     0x2629 _build/nrf52832_xxaa_nrf_drv_uart.c.o
 .debug_line    0x0000000000006236      0x7d1 _build/nrf52832_xxaa_system_nrf52.c.o

.debug_str      0x0000000000000000    0x6b8d6
 .debug_str     0x0000000000000000    0x60aa9 _build/nrf52832_xxaa_main.c.o
                                      0x615e6 (size before relaxing)
 .debug_str     0x0000000000060aa9      0x248 _build/nrf52832_xxaa_gpio.c.o
                                      0x61820 (size before relaxing)
 .debug_str     0x0000000000060cf1     0x7c97 _build/nrf52832_xxaa_nrf_drv_gpiote.c.o
                                      0x690af (size before relaxing)
 .debug_str     0x0000000000068988     0x1358 _build/nrf52832_xxaa_nrf_drv_timer.c.o
                                      0x68a02 (size before relaxing)
 .debug_str     0x0000000000069ce0     0x1806 _build/nrf52832_xxaa_nrf_drv_uart.c.o
                                      0x693b6 (size before relaxing)
 .debug_str     0x000000000006b4e6      0x3f0 _build/nrf52832_xxaa_system_nrf52.c.o
                                      0x5c3af (size before relaxing)

.debug_loc      0x0000000000000000     0x670c
 .debug_loc     0x0000000000000000     0x29ec _build/nrf52832_xxaa_nrf_drv_gpiote.c.o
 .debug_loc     0x00000000000029ec      0xb56 _build/nrf52832_xxaa_nrf_drv_timer.c.o
 .debug_loc     0x0000000000003542     0x31ca _build/nrf52832_xxaa_nrf_drv_uart.c.o
